:1000000000308A00E02B0000FF00030E8301A100F6
:100010007F08A0000A08A8008A01A00E0408A20018
:100020007708A3007808A4007908A5007A08A6003C
:100030007B08A700831383128C308400801C222845
:100040008C186F288B1E26280B1962282208840022
:100050002308F7002408F8002508F9002608FA000C
:100060002708FB0028088A00210E8300FF0E7F0E60
:1000700009000A108A100A1182078734FF340A1017
:100080008A100A11820707340F34003407340F3402
:10009000023407340F34043407340F34083407347F
:1000A0000F34103407340F34203407340F34053440
:1000B00007340F3409340A108A100A1182070934F0
:1000C00002340034AD0B6C281930AD00AE0A29148F
:1000D0003B082E020319A9110B118A112628291D8C
:1000E0007628851D75288511762885158C108A112E
:1000F000262847308400000803198C280130F800B6
:10010000F701F70B8128F80B80280E30F700F70B6A
:1001100087280000800B7E2800341930AD00AE0126
:10012000AF010130B800A915FF30BE0000348501D1
:10013000860112306500FF3066008316811383123A
:100140008D2081010630F700F71DAE2807308101B0
:10015000813084000008C0390F388000640081308D
:1001600084000008C039770480008B160030F80046
:10017000053892009430831692008C14C03083129C
:100180008B048515052CF801F901F701FA014A08DD
:10019000031DCD2849080319E7281030CB000310B0
:1001A000C70DC80DF70DFA0D4A087A02031DDA28AB
:1001B00049087702031CE3284908F702031CFA03E5
:1001C0004A08FA020314F80DF90DCB0BCF280000F2
:1001D00000341030F700FA01CD01CA0CC90C031C21
:1001E000F7284B08FA070318CD0A4C08CD07CD0CA9
:1001F000FA0CF90CF80CF70BED2800342E083E022F
:10020000031C2D290330C800E830C700CA01330899
:10021000C900C3207908C8007808C7007908CA0057
:100220007808C900CC014608CB00E9207908B50060
:100230007808B4003508FA0034080319B503B4038C
:10024000C7007A08C800C708031D2929C808031970
:100250002D290130C70079201A2900342E083E02CA
:10026000031C60290330C800E830C700CA01330806
:10027000C900C3207908C8007808C7007908CA00F7
:100280007808C900CC014608CB00E9207908B50000
:100290007808B40029153508FA0034080319B503A5
:1002A000B403C7007A08C800C708031D5A29C80844
:1002B00003195E290130C70079204B2929118511C6
:1002C0000034C508031D67290530C600FE20450817
:1002D000803C03187A294508013C03187A29031049
:1002E000C50C031C76293308C6002E210130C60038
:1002F000FE206B294508013C031890290310C50C0A
:10030000031C89290330C6002E210130C600FE20BF
:100310008F290130C6002E210130C600FE207A2927
:100320000230C600FE2000340730C600FE20AA01BD
:100330002A0883169B009C131C141A08FF3C0319FF
:10034000AF2983122A0883169B009C131C141A08D9
:100350008312C200C5006121AA0A9829831683125C
:1003600000340A30B30005150730C600FE202230E5
:10037000C500612194210511AA010514051ABE29A1
:1003800005100608FF3AAC002C08013A0319CF29E2
:10039000813A03190B2A7F3A0319482A612AAB01D3
:1003A0002B08023C031C0A2A2B085B20C2002A08E7
:1003B00083169B008312420883169A001C15831231
:1003C0000B08F7008B13831655309D00AA309D0053
:1003D0009C149C18E9291C11770883128B040130A6
:1003E0002A07C20083169B00FF309A001C15831257
:1003F0000B08F7008B13831655309D00AA309D0023
:100400009C149C18012A1C11770883128B04AA0AD9
:10041000AB0AD029922AAB012B083920FF3C0319E3
:10042000472A2B083920C2002A0883169B00831212
:10043000420883169A001C1583120B08F7008B13D1
:10044000831655309D00AA309D009C149C18262AC6
:100450001C11770883128B0401302A07C20083160F
:100460009B00FF309A001C1583120B08F7008B13BA
:10047000831655309D00AA309D009C149C183E2A7E
:100480001C11770883128B04AB0AAA0A0C2A922A41
:100490002A0883169B0083122C0883169A001C15C9
:1004A00083120B08F7008B13831655309D00AA307A
:1004B0009D009C149C185A2A1C11770883128B04E7
:1004C000922A2A0883169B0083122C0883169A000E
:1004D0001C1583120B08F7008B13831655309D00F3
:1004E000AA309D009C149C18732A1C117708831253
:1004F0008B0401302A07C20083169B00FF309A004C
:100500001C1583120B08F7008B13831655309D00C2
:10051000AA309D009C149C188B2A1C11770883120A
:100520008B04AA0A0515942105112C0FBD29082C4E
:10053000F701F801420803104318F707F70CF80C0D
:10054000C318F707F70CF80C4319F707F70CF80C6A
:10055000C319F707F70CF80C431AF707F70CF80C58
:10056000C31AF707F70CF80C431BF707F70CF80C46
:10057000C31BF707F70CF80C00340608AC00FF307B
:10058000AC062C08F839B000B00CB00CB00C1F3021
:10059000B005301ECD2A0310B00D3008C200033064
:1005A000C30098227808B0002C080739B6003C3008
:1005B000BB003608043C031CE22A0530B7000130BA
:1005C0003607B9003608053C031DEB2A0130B70099
:1005D000B9017830BB003608053C0318F82A360804
:1005E000073C031CF82A0230B70005303602B90078
:1005F000092C01303B02BD000230C8005830C70052
:10060000CA013B08C900C3207808BF008D20B10192
:100610000130BA000A2C3B082E02031C1A2B3B089F
:10062000AE02AF0AB80A380837020318192B013096
:10063000B800A9153F082F02031C222BAF01B108F7
:10064000031DB10300340230A906A918292B051097
:100650002A2B0514851C2A2B8D203008B10039085F
:10066000BA00132CB1080319742B1930B3000B23F3
:10067000003029180130013C031D462B0230A90629
:10068000A918442B0510452B05142910B10803198E
:10069000712B3108063C031C712B30083102031802
:1006A000712B39083802031D712BAE08031D712B05
:1006B000851105150730C600FE20AA012A08023C54
:1006C000031C6F2B3908C2000330C30098222A088C
:1006D00078073F20C400C5006121AA0A5E2B0511DE
:1006E0008515B108031D372B0510142C8D200B2305
:1006F00038083A0203197F2BBA08031DDE2B00309D
:10070000A9190130013C031DDE2B051585110030B0
:10071000A91A0130003A031DA72B1930B3002E0887
:10072000AB0083169B019C131C141A08FF3C031991
:100730009F2B831294210330C600FE208316831260
:100740002B083D07F8002E087802BC00A9160A30D5
:10075000B3003C08BE003C082E020318C52B07302E
:10076000C600FE20AA012A08023C031CC42B39083B
:10077000C2000330C30098222A0878073F20C40033
:10078000C5006121AA0AB32BAB2B3B08BE00193070
:10079000B30083169B019C131C141A08FF3C031919
:1007A000D42B83129421831683123D082E02031842
:1007B000DB2B8316D42B05118515A911772B152C4E
:1007C00084011F30830507309F002910A9102911CB
:1007D000A9112912A912AA01AB01AC01AD01AE0108
:1007E000AF01B001B101B201B301B401B501B6016D
:1007F000B701B801B901BA01BB01BC01BD01BE011D
:10080000BF010130C70079209728051A082CB129AB
:10081000BD2AF92A8518132C2E08023C031C122C21
:0C0820000B230C2C232B322B762B6300B7
:0A42000006000A0009001400FF0088
:02400E00613F10
:00000001FF
